:020000040000FA
:100000008316FF3085009F01053081009516151677
:1000100096168312073099008B1520308400DF007C
:100020008001840ADF08031D10289320B33081006B
:100030000B110A30B0007C20031D2028A50A1B28C4
:100040000F21A6002502031828280301A60000217D
:100050002608240603192E287C2028285E20A020AC
:100060000030051EFF308500C10041128316F830B4
:10007000850083123B28C00F4128410885000B19D9
:100080001521C108031D512840083707031805151D
:100090004008350703188514400833070318051472
:1000A0003B28400837070318051140083507031897
:1000B000851040083307031805103B287820A70057
:1000C000013E0319732827308400840AA20A031909
:1000D000A30A782080002B300406031D6528A20A9D
:1000E0000319A30A08002008A2002108A3005E2823
:1000F00023088A00220882009C20013E03198528DB
:100100000530A0070318A10A7C28A40AA00A031935
:10011000A10A9C20013E031993282008A20021086F
:10012000A30003010800A4010130A100A30077305F
:10013000A000A200FF38080021088A0020088200E1
:100140002808B1002708AF00031DAE282908B30016
:100150002A08B5002B08B700BF0108000730BF0010
:100160000130B200B400B600330829020318BB28DE
:10017000B203B203003CB80035082A020318C328B2
:10018000B403B403003CB90037082B020318CB2892
:10019000B603B603003CBA00380839020318D72862
:1001A00038083A023A080318DC283808DC283908ED
:1001B0003A023A08031C3908003CBE00BB00BC00F0
:1001C000BD0008002408002141088500831605129F
:1001D0008312851EE9280F30F82005080B106300F4
:1001E00000005A30F820851AE928851EF5280028D5
:1001F00081010B110B1DFA28FF3E031DF828080092
:100200008512831685129A009B018C131C1555309C
:100210009D00AA309D009C14851683120800831649
:100220009B011C141A08831208000108B33E8100C8
:100230000B11AE0803192229AD0B2229AE0B22297E
:1002400024080021851A2829AC0A0319E228392933
:10025000FC302C0703182E29AC0139297C205E20A4
:10026000B301B501B701A0200A30B000AC010830DD
:10027000AE00BF0803196B29AF0B08002708AF00B9
:1002800029083306031D46293F104E293808BB07AD
:10029000031C4E293E08BB073208B3072A0835065F
:1002A000031D5429BF105C293908BC07031C5C29B5
:1002B0003E08BC073408B5072B083706031D622922
:1002C0003F1108003A08BD07031C08003E08BD079F
:1002D0003608B7070800B10803197429B00B0800E5
:1002E0000A30B000B10B08005E20A02008000034E6
:1002F0000534FF3400340034013400340034003459
:100300000034003405340034FF3400340134003448
:100310000034003400340034053400340034FF3439
:1003200001340034003400340034FF34023401342A
:10033000FF3400340034023401340034FF3400341C
:100340000234013400340034FF34FF340234013409
:10035000FF34403400340234013440340034FF347C
:10036000023401340034FF344034FF340034FE34AE
:10037000FF3400340034FF340034FE340034FF34E2
:100380000034FF340034FE3400340034FF34FF34D2
:100390000034FE34F0340034F034FF340034FE34E2
:1003A000FF349B340034FF340034FE34F034F03436
:1003B000F034FF340034FE34803480348034FF3431
:1003C0000034FE34303430343A34FF3400340134F5
:1003D000FF3400340034003401340034FF3400347E
:1003E0000034013400340034FF34FF34033400346B
:1003F00080348034803400340134C834FF34FF3416
:100400000034013400340034003400340134C83482
:10041000FF34FF340034013400340034003400343D
:100420000134C834FF34FF34003401340034003464
:10043000003400340134C834FF34FF340034013454
:1004400000340034003400340134C834FF34FF3445
:100450000034013400340034003400340134C83432
:10046000FF34FF340034013480348034803402346B
:100470000234003400340034FF3406340A34FF34CC
:100480000034003406340A34FF34FF3400340634B8
:100490000A340034FF34003406340A340034FF34A4
:1004A000FF3406340A3400340034FF3406340A348E
:1004B000FF340034FF34FF341934FE34FF34003489
:1004C00000341934FE34FF34FF3400341934FE3460
:1004D0000034FF3400341934FE340034FF34FF3468
:1004E0001934FE3400340034FF341934FE34FF3440
:1004F0000034FF34FF3404340A34FE342034003432
:1005000004340A34FE348034003404340A34FE34B3
:10051000F034003404340A348034F0340034FF34CE
:1005200004340A3400341034FF3404340A34003400
:100530008034FF3404340A340034F034803404341A
:100540000A3410341034F03404340A34F0341034E3
:10055000F03404340A3440340034FA34FF340A34BA
:100560000434F0340034F0340A34043420340034D9
:10057000F0340A3404348034003480340A340434CF
:10058000F03400342034FF340034053400340034B7
:100590000A3400340534003400340034FF34FF34AE
:1005A000723467346234733461345F3469346E3466
:1005B000653474342E34613473346D342034303403
:1005C00039342F34303436342F34323430343034FC
:1005D00037342034523432342E3430342E343234E2
:1005E0002834633429342034503465347434653409
:1005F0002034473472346934663466346934743470
:1006000068347334203432343034303436342D345A
:100610003234303430343734203472346734623416
:1006200073346134403470346534743465347334F5
:1006300077346F3472346C3464342E3464346534FB
:100640006D346F346E342E3463346F342E3475341D
:020650006B3409
:02400E00E43C90
:00000001FF
